:100000004EC168C1E6C266C165C1C9C463C162C1EF
:1000100061C160C15FC15EC15DC15CC15BC15AC1EC
:1000200059C158C157C15A03680061006600740085
:100030006D0061006E006E00230073006F006600AB
:1000400074007700610072006500200028007700CE
:10005000770077002E00740075002D0063006800A3
:1000600065006D006E00690074007A002E00640067
:1000700065002F007E0068006500680061002900AF
:100080003A034800490044002D0044007500720006
:100090006300680066006C007500730073006D00FB
:1000A0006500730073006500720020002800500096
:1000B0006E0050005300410029003A0368006500BB
:1000C000680061004000680072007A002E00740031
:1000D00075002D006300680065006D006E0069000A
:1000E00074007A002E00640065003A003000300091
:1000F000300033001201100100000008C016D9279B
:100100000001010203010902220001010080FA0935
:100110000400000103000000092101010001228AFE
:1001200000070581030800100600FF0901A10195E1
:10013000017510A4A18016C00026C0033504451423
:1001400055FD67010010000944790481020B480045
:10015000010055FD6731F0F000C7010001000945BD
:100160007908B103C0150027FFFF0000350047FFE5
:10017000FF00005506653109817907810A26FF03D2
:1001800009457905A18246FF0A55056721D1F0008E
:10019000098581020986B102C0094479068102B449
:1001A00025017501091FA1020982B1029507B1035A
:1001B000C0C00603070409042C0356006F006C003E
:1001C00075006D0065006E007300740072006F00B2
:1001D0006D00200069006E0020004E006D00B3002D
:1001E0002F00680028035300700065006900730049
:1001F00065007300700061006E006E0075006E0097
:100200006700200069006E002000560028034500AA
:1002100078007400720061002D00530070006100CE
:100220006E006E0075006E006700200069006E00B1
:10023000200056003003470065007A00E4006800A3
:100240006C00740065007300200056006F006C00A5
:1002500075006D0065006E00200069006E002000D2
:100260006D00B3003A039A9989406666E63F3333DE
:10027000C340000030416666D64000006041CDCCEE
:10028000FC400000904133330B410000C0416666E2
:100290002E4100000C4266668A410000874211240C
:1002A0001FBECFE5D4E0DEBFCDBF10E0A0E6B0E0DA
:1002B000E6EDFCE002C005900D92A037B107D9F73A
:1002C00010E0A0E7B0E001C01D92AB3AB107E1F742
:1002D00015D400C595CE8BB780688BBF8BE4809317
:1002E00080008AE580937F0008951F93CF93DF936A
:1002F00060919100635067FDC9C080918D00C1EA93
:10030000D0E0C81BD10980918C008D3209F0A8C0C3
:10031000683009F0B5C083EC809374008AE580935F
:100320006000109270008881807619F0CE0191D320
:1003300083C09A8110927D008981882321F41092D4
:100340007E0082E073C0853019F4909392006DC0F6
:10035000863009F056C08B81813041F484EF90E003
:100360009093900080938F0092E146C0823041F4D8
:1003700086E091E09093900080938F0092E23CC0E1
:10038000833019F5992341F482EB91E0909390002A
:1003900080938F0096E030C0913041F486E290E087
:1003A0009093900080938F009AE526C0923019F4C4
:1003B00080E890E004C09330E1F48AEB90E0909301
:1003C000900080938F009AE317C0813241F486E455
:1003D00091E09093900080938F0099E00DC082325D
:1003E00041F488E291E09093900080938F009AE826
:1003F00003C0CE01F0D2982F80E480937000892F43
:100400001BC0883021F481E024E930E011C089303C
:1004100019F49093940009C08A3011F481E006C069
:100420008B3019F48BE48093800080E02DE730E07E
:100430003093900020938F00982F8F3F39F488815C
:1004400087FD9E8180E88093700007C08F8188239C
:1004500021F48E81891708F4982F9093610010C0C1
:100460008091700087FF0CC0CE01E0D28F3F21F455
:100470008EE18093600004C0882311F01092610027
:1004800080919100181614F41092910080916000F0
:1004900084FF46C0609161006F3F09F441C09091B4
:1004A0007400693008F047C01092610088E898270E
:1004B00090937400662309F447C020918F00309117
:1004C00090008091700086FF0AC0962FF901A5E781
:1004D000B0E084918D9331969150D9F708C0962F52
:1004E000F901A5E7B0E081918D939150E1F761505A
:1004F000C901860F911D6F5F0196909390008093C4
:100500008F007727162F85E790E05FD01C5F1C30A7
:1005100010F01CE003C08FEF809361001093600027
:1005200094E180B38C70B1F49150D9F7109292009D
:1005300010928B000FC068506093610088E8982784
:100540009093740068E0B9CF60E085E790E03DD01B
:1005500014E0E1CFDF91CF911F9108951F93DC014B
:10056000162F80917F0084FF07C08091800098E85B
:1005700089278093800003C08AE580937F00912FB4
:10058000E1E8F0E08D91819391501916DCF3612F31
:1005900081E890E01AD01C5F10937F001F910895AE
:1005A000A82FB92F80E090E041E050EA60956F5F9E
:1005B00058F42D9138EF82279795879510F084276E
:1005C00095273F5FC8F3F3CF0895EADF8D939D939E
:1005D0000895CF93CFB7CF93C395839BE9F7839BC0
:1005E0001DC0839B1BC0839B19C0839B17C0839B2B
:1005F00015C0C0918E00C395C0938E00DF93DD2798
:10060000C2B7D2BFC85CD1B7C23012F0D15003C05C
:10061000CF3F0AF4D395D1BFDF913EC1DF93C091A4
:100620008D00DD27CB56DF4F839B02C0DF91D7CFF4
:100630002F930F931F9320E8839921604F933F934B
:100640000F92839922601FEF3BE0022F220F00C020
:1006500083990C602027087040B311F4000036C065
:10066000B4C043FFC89540B3206800000227839BB5
:100670000AC0287F11F040B388C040B31E7F839B1F
:10068000829901C06AC043FDC89540B321604C7097
:10069000839908C0B9F3217F40B309F087C01D7F5B
:1006A00000C000C043FFC89540B322600000839B98
:1006B00008C0237E11F040B387C040B31B7F00C049
:1006C00000C043FDC89540B324600993839908C0D6
:1006D000277C11F040B387C040B3177F00C000C033
:1006E00043FFC89540B32860012F839B08C02F7833
:1006F00011F040B387C040B30F7E00C000C043FD7F
:10070000C89540B320611FEF839908C02F7111F085
:1007100040B387C040B30F7D00C000C043FFC89501
:1007200040B32062315038F0839B08C02F732230D1
:1007300040B314F085C08EC00F7BC89543FDC895AB
:1007400040B32064000083998CCF2F77243040B3CE
:100750000CF00AC00F77000084CF09937DC043FDE1
:10076000C89540B320680000022783990AC0287FFB
:1007700011F040B38CCF40B31E7F839B829901C0A0
:10078000ECCF43FFC89540B321604C70839B09C0F8
:10079000217F19F040B300008ACF40B31D7F00C015
:1007A00000C043FDC89540B3C1F22260839908C0E0
:1007B000237E11F040B389CF40B31B7F00C000C03F
:1007C00043FFC89540B324600993839B08C0277CEE
:1007D00011F040B389CF40B3177F00C000C043FD84
:1007E000C89540B32860012F839908C02F7811F075
:1007F00040B389CF40B30F7E00C000C043FFC8950F
:1008000040B320611FEF839B08C02F7111F040B3EC
:1008100089CF40B30F7D00C000C043FDC89540B3F1
:1008200020623150B8F0839907C02F73223040B353
:100830000CF089CF0F7BC89543FFC89540B3206467
:10084000839B8DCF2F77243040B30CF00FCF0F77E1
:10085000000085CF002717C03B503195C31BD04007
:100860000881033CE9F00B34D9F020918B00198109
:10087000110F1213EFCF4A81441F093631F10D32A7
:1008800011F0013E39F7009393000F903F914F9183
:100890001F910F912F91DF91CF91CFBFCF911895DD
:1008A00020919300222389F310919100112369F57F
:1008B00034306AF13093910020938C0010918D00B8
:1008C0003BE0311B30938D0022C00091910001303C
:1008D000E4F40AE54F7049F43091600034FD18C02B
:1008E00000936000C4E7D0E017C030917F0034FD72
:1008F0000FC000937F00C0E8D0E00EC0279598F4A9
:10090000415099F4220F0000F9CF3AE501C032EDD1
:10091000032EC0E0D0E032E011B31C60939A11BB0B
:1009200002B320E41CE0012746E002BB279520F437
:10093000415021F4220FF9CF012746E000000000CA
:100940003B5A02BBD8F2279528F4415029F4220FD4
:100950000000F9CF012746E0279502BB20F4415063
:1009600021F4220FF9CF012746E02991000033231B
:1009700002BB21F6037F10919200110FC250D040AC
:1009800002BB11F010938B00086011B3137F402F4E
:10099000437FC895C89502BB11BB42BB76CF2FB62B
:1009A0003090640033943092640029F430906500F4
:1009B0003394309265002FBE1895982F8091710066
:1009C000882321F49093730084B314BA9093720037
:1009D000909371000895FC018381833021F5828119
:1009E000863091F0873028F4843041F08530D9F496
:1009F00008C0873061F08830B1F40CC0E8EBF1E05A
:100A00000BC0E4EEF1E008C0ECE0F2E005C0E4E386
:100A1000F2E002C0E4E6F2E0F0939000E0938F0091
:100A200084919927089580E090E00895FC01653055
:100A300069F48281938124E08030920720F49093BE
:100A40006D0080936C00848180936E0081E090E063
:100A50000895FC0180818076803211F5818181309A
:100A6000B9F48381813049F482E690E0909390005C
:100A700080938F0088E090E00895833089F48AE6BF
:100A800090E09093900080938F0085E090E008952F
:100A9000893031F48381833019F48FEF90E0089529
:100AA00080E090E00895DC0108D1802D681729F0DE
:100AB0006DBBF894E29AE19A78940895EF92FF92D0
:100AC0000F931F93CF93DF937C018B01EA01452B9A
:100AD00071F0E1990CC0F7016081C801E4DF219752
:100AE00031F00894E11CF11C0F5F1F4FF2CFDF9132
:100AF000CF911F910F91FF90EF900895CF93DF93C7
:100B0000CDB7DEB722970FB6F894DEBF0FBECDBFCC
:100B100080E885BF8FEC81BFDEDB789480E888B900
:100B20008AEF88BB84E087BB80E585BB80E384BB1C
:100B300083E282BB82E181BB22E0A0E0B0E0FE0163
:100B40003196122EC2D089819A813FEF8F3F930751
:100B500021F090936D0080936C00E4E6F0E0A2E059
:100B6000B0E0122EB2D083E083BF8AE088BD81E27C
:100B70008FBD89EC8EBD80E289BF83EC87B987EC9D
:100B800086B900E001C0012F10918E00AEDB3699CE
:100B900058C024B135B187B19927877090708130E2
:100BA000910539F0039759F4309363002093620064
:100BB00004C0309369002093680082EC3FC048B5C0
:100BC000C90195958795959587958C3910F051EECB
:100BD00002C0582F5A5B80916C0090916D002817CD
:100BE00039074CF480916600909167008217930753
:100BF00084F04F5F0EC0C2968217930714F44AE048
:100C000008C08091660090916700281739070CF0A2
:100C100041503093670020936600852F451708F4F4
:100C2000842F8A3008F48AE088BD82B390E1892756
:100C300082BB949B02C083EC01C081EC87B987EC36
:100C400086B9101709F4A0CF20917100222391F0EA
:100C500080917300815031F484B390E1892784BB83
:100C600080917200922F915009F4A49A9093710090
:100C70008093730080917F0084FF04C068E082E667
:100C800090E06CDCE1997FCF80916E0080FF02C024
:100C900062E401C060E084E090E005DF42E050E003
:100CA00060E070E08CE690E009DF42E050E062E056
:100CB00070E084E690E002DF66CFE199FECFBFBB33
:100CC000AEBBE09A11960DB20895F7DF01921A9427
:060CD000E1F70895FFCFDB
:100CD6005AFF0080008000800000DA0AB20200009D
:00000001FF
